S018000064656D6F70726F675F7333326B3134342E7372656374
S1132000007000209D2D00002B2B00005F2E00008F
S1132010872E0000932E0000D52E00000000000043
S1132020000000000000000000000000D72E0000A7
S1132030D92E000000000000DB2E0000912A0000D1
S1132040CD2E0000CD2E0000CD2E0000CD2E0000A0
S1132050CD2E0000CD2E0000CD2E0000CD2E000090
S1132060CD2E0000CD2E0000CD2E0000CD2E000080
S1132070CD2E0000CD2E0000CD2E0000CD2E000070
S11323F0CD2E0000CD2E0000EE11AA55FFFFFFFFE9
S1132400FFFFFFFFFFFFFFFFFFFFFFFFFE7FFFFF59
S113241080B500F00DF800F061F901BD80B500F061
S113242065F800F021FA01BD80B500F0F4FA01BDB1
S113243082B06846DFF89814D1E90023C0E900238C
S1132440DFF89004016831F080410160016851F0C7
S113245084410160DFF880140868C0F3022000287A
S113246004D10120020212F4E0620A60DFF86C1465
S1132470DFF86C241268D20701D4DFF868146A46C6
S1132480105CB1FBF0F04FF46141B0FBF1F0C01D02
S1132490C008C004C00C80B2C004C00C50F0E0609E
S11324A0DFF844140860DFF84404DFF844140860DB
S11324B0DFF84004002101600021DFF83C241160B2
S11324C00021DFF838241160DFF834145FF470322F
S11324D00A600A6852F088020A600121DFF82424A5
S11324E011605FF44021016002B0704770B5DFF8FD
S11324F018442078002818D1DFF81054280000F080
S11325003CF8012838D12878002835D0287841288B
S113251032DA00F0BAFADFF8F8130860012020700C
S11325200020DFF8F013087026E0DFF8E863DFF836
S1132530DC5330782844401C00F01FF8012811D1E6
S11325403078401C307030782978884214D10020CB
S113255020706878FF280FD1A87800280CD1FFF7E5
S113256063FF09E000F091FADFF8A413096864310D
S1132570814201D20020207070BD02000020DFF8EB
S113258070130968C1F34051002904D0DFF88803AF
S1132590006810700120C0B27047FCB403006846A4
S11325A0DFF87843D4E90056C0E90056DFF87043F9
S11325B02068C0F30220002804D10120050215F48C
S11325C0E06525604FF4FA546D46285CB4FBF0F5E1
S11325D0002600E0761C3000C0B2122825D2D14F6C
S11325E0180080B23400E4B217F824406043B5FB0D
S11325F0F0F400FB14500028ECD11C00A4B230000D
S1132600C0B217F820004443B5FBF4F008800888F2
S11326100028DFD0088840F20114A042DAD2F6B2D2
S113262057F826001060012000E00020F6BC704737
S113263038B5BD4D286850F080402860286850F0B7
S11326408050286000F021FA0400FA342868C001A0
S113265003D400F01AFA8442F8D231BD38B5B24D31
S1132660286830F080402860286830F08050286066
S113267000F00BFA0400FA342868C00103D500F016
S113268004FA8442F8D231BD38B5A74D2868002831
S11326900ED4286850F00040286000F0F6F90400D9
S11326A0FA342868C00203D400F0EFF98442F8D267
S11326B031BD38B59C4D286800280ED5286820F017
S11326C00040286000F0E1F90400FA342868C002F0
S11326D003D500F0DAF98442F8D231BD7CB500208C
S11326E0ADF8040004220021684600F0E1F940F24C
S11326F067658E48016851F080410160FFF7D9FF9A
S1132700FFF796FFFFF7C0FF894C206830F40050B4
S11327102060FFF7CEFFFFF78BFF6A4601A94FF455
S1132720FA70FFF73AFF21684FF678700140216094
S11327302068BDF80410491E50EA0160206020683A
S11327409DF80110491E11F007010843206020681C
S11327509DF80210491EC90411F460110843206059
S113276020689DF80310491E090411F4E021084370
S113277020609DF80200042802DA9DF8020000E0BF
S113278004202168C0B2401E800510F440000843B4
S11327902060206850F080002060002006E00021C6
S11327A0644A03009BB242F82310401C010089B222
S11327B08029F4D3002006E000215F4A03009BB285
S11327C042F82310401C010089B22029F4D3564E4C
S11327D03068C009C00150F01F003060306850F408
S11327E000303060306850F480303060306830F051
S11327F0005030607FF020405049086050485FF03E
S113280080610160002D0AD525F00045016851F46E
S11328100011016025F060454A48056004E0AD04FC
S113282025F06045474805600020474908605FF08F
S1132830FF3046490860464846490860306830F42D
S1132840000030602168444801402160FFF706FF22
S113285000F01BF90400FA343068000103D500F0DD
S113286014F98442F8D273BD7CB5384801688905EF
S11328702DD533490968090C11F00F01374A00239B
S11328800FE01C00E4B2A408A400E41C1D00EDB297
S113289015F00305641B145D6D461E00F6B2AC55BD
S11328A05B1C1C000D00E4B2EDB2AC42E9D34FF462
S11328B0007202602A4800682A4A10609DF80000ED
S11328C0FF2804D1C9B2022901D1FFF7ADFD73BDC0
S11328D0B42E0000AC5106400442064000127A00B7
S11328E00842064080841E0010B0064000C01FC08D
S11328F014B0064018B0064020B0064024B006408C
S113290028B006402CB006405500002000000020EE
S113291044000020540000201CB00640BC2E0000DF
S113292004410640F42D000000400240905006404F
S1132930044002408040024080480240A4480240D3
S113294010410240144102402840024030400240FD
S113295006003B0020400240F7EFFFFF1841024011
S113296008400240480000202F48016851F47001DB
S113297001602E48016831F0804101602C482D49E6
S11329800160006842F220102B4908604FF6FF7086
S11329902A490860704710B40023012028490A68B6
S11329A0C2F30342521C0968090E11F00F010129F8
S11329B006D0022906D003290CD0062912D020E023
S11329C0204B1FE02049096811F00101002900D0C3
S11329D01C4B17E01D49096811F003011C4B53F807
S11329E021300FE017491B4C2368C3F302235B1CFF
S11329F02468C4F30444103461435B00B1FBF3F373
S1132A0000E00020C0B2002803D0B3FBF2F012496A
S1132A10086010BC7047114A116889B2104801431C
S1132A2051F004011160704788ED00E034EF00E0DC
S1132A300420054020C528D9002005400820054071
S1132A401040064000127A0008420640084306403F
S1132A50C82E0000084606400084FF1F0CED00E06D
S1132A600000FA050D4800684FF47A71B0FBF1F0EC
S1132A70401E0B49086000200A49086007200A49E3
S1132A8008600020094908607047084800687047DA
S1132A9006480168491C0160704700000084FF1F5C
S1132AA014E000E018E000E010E000E05000002036
S1132AB010B5044610460A460146204600F002F8C6
S1132AC0204610BD62F30F2262F31F42401810F03B
S1132AD0030308D0C91A1FD3DB0748BF00F8012D30
S1132AE028BF20F8022D130030B4144615461039BF
S1132AF028BF20E93C00FAD8490728BF20E90C0088
S1132B0048BF40F8042D890028BF20F8022D48BF93
S1132B1000F8012D30BC7047C91818BF00F8012D0A
S1132B20CB0728BF00F8012D7047FEE780B500F001
S1132B3007F8FFF76DFC00F09DF8FFF76FFCFAE76C
S1132B4080B500F029F83248016851F080410160F5
S1132B503048016851F0804101602F48016851F00C
S1132B60804101602D48016851F4007101602C48D6
S1132B70016851F4007101602A48016851F4A061B0
S1132B8001602948016851F4A0610160FFF76AFF00
S1132B9000F060F862B601BD10B540F2011123489F
S1132BA001602420224A1060224802681202FBD4E9
S1132BB0012202600268D201FCD51F4A106800029B
S1132BC0FBD410684008400010601C4B1C6840F2A5
S1132BD0023004431C605FF4C010194B1860106885
S1132BE00002FCD4106850F0010010601068C001AD
S1132BF0FCD514480160144814490860144800685E
S1132C00C0F303600628F9D1FFF7C5FE10BD00002C
S1132C102C510640305106403451064018B004404F
S1132C201CB0044010D0044014D0044004410640B9
S1132C30084106400041064000460640044606405E
S1132C4008460640044206401200010614400640AD
S1132C50104006401648016851F48071016015481F
S1132C60016851F0010101601348016851F001014C
S1132C700160704780B5FFF708FF104A1168411AD8
S1132C80B1F5FA7F13D30E4B1978002907D101212E
S1132C9019700C490B6853F001030B6006E0002126
S1132CA0197005490B6853F001030B60106001BDF6
S1132CB000C00440D4F00F40C4F00F404C0000208A
S1132CC056000020C8F00F402DE9F043244B254E58
S1132CD0254F264CDFF898C0DFF898E0264DDFF842
S1132CE09C8027482749284A05E096F8009083F8F5
S1132CF000905B1C761CB742F7D1E64509D09CF8DE
S1132D0000302370641C1CF1010CF6E700232B70C7
S1132D106D1CA845FAD18A4204D00B780370491C73
S1132D20401CF8E70021194A194B934210D00020A7
S1132D3004E052F8204043F82040401C154CB0EB0E
S1132D40940FF6D31448C9B250F82100036004E08C
S1132D501148C9B250F821000260BDE8F08300BFF9
S1132D600084FF1FD02E0000D42E00000484FF1F17
S1132D70DC2E0000DC2E00000000002057000020A4
S1132D80000000000000000000000000002000001F
S1132D900080FF1F00040000C42E000072B6002152
S1132DA0002200230024002500260027B846B94647
S1132DB0BA46BB46BC460A490A4A521A013A05DDDC
S1132DC00020042308601944043AFBDA06488546C7
S1132DD0064880470648804762B6FFF7A7FEFEE72D
S1132DE00080FF1FFF6F0020007000206929000091
S1132DF0C92C000008030202090303020A030303A7
S1132E000B0403030C0404030D0504030E0504045E
S1132E100F0604041006050411070504120705052E
S1132E2013080505140806051508070516080706FE
S1132E301708080618080807190808084EF68851E4
S1132E40CEF20001086840F470000860BFF34F8FB1
S1132E50BFF36F8F4FF00070E1EE100A7047FEE78A
S1132E6000F00DF8002801D0AFF30080AFF300802C
S1132E700020AFF30080FFF759FE00F002F80120B4
S1132E80704700F001B8FEE70746384600F002F844
S1132E90FBE7FEE780B5AFF30080024A110018207B
S1132EA0ABBEFBE726000200AFF30080FFF7C6FFCE
S1132EB0FFF7D6FF000102040810204000010204BD
S1132EC00810204008ED00E0006CDC02FFF7FEBFB4
S10F2ED0006CDC02FEE7FEE7FEE7FEE714
S9032EA925
